:100000000C94240018950000189500001895000025
:100010000C94871B18950000189500001895000097
:10002000189500000C944104189500000C94DB1BFB
:100030000C94FD1B18950000189500001895000001
:1000400018950000189500008FE181BD87E181BD02
:100050008FE58DBFC2E2E0E04E2E84E08EBFD4E09B
:10006000F4E05F2EEEEFF3E0A0E6B0E088278D939A
:100070003197E9F789E189B980E080BD88E18AB9E3
:1000800066248FEF87BB8FEF8BBB8DE181BD85E150
:1000900081BD579A86B1856086B985E083BF80E0CF
:1000A00080930E0189B7816089BF8FEF93E09BBD7C
:1000B0008ABD8FEF93E099BD88BD83EF8FBD81E04E
:1000C0008EBD80E381BB88E082BD85E085BD89B7B8
:1000D000806489BF81B5886181BD81BDA0E9B0E040
:1000E0008C918F778C93A0E9B0E08C918F7B8C936F
:1000F000E3ECF1E0A3E9B0E00E94CF1CA3E9B0E09B
:100100008C9181FBA0E9B0E08C9185F98C93AAE4F5
:10011000B0E08D919C91A2E0B1E08D939C93A8E416
:10012000B0E08D919C91A4E0B1E08D939C9381E02F
:1001300080939F0081E080939300009193000630AC
:1001400018F011F00C94C200E3E9F0E0A190BB2498
:10015000EAEEF1E0AA0CBB1CEA0DFB1DA3E9B0E03E
:10016000AD90BB24ACEEB0E0AA0CBB1CAA0DBB1D2D
:100170000E94D11CA3E9B0E08C918F5F8C9311F0A9
:100180000C949D007894A8950E94CE1AA2E9B0E044
:100190008C93E3ECF1E0A3E9B0E00E94CF1CA0E96E
:1001A000B0E08C9185FBA3E9B0E08C9181F98C9350
:1001B00040919300E3ECF1E0BB27A0E10E94CF1C4B
:1001C000041711F40C94EA00E3ECF1E0A3E9B0E0C9
:1001D0000E94BC1C009192000D3011F00C94F900AB
:1001E000A0E9B0E08C9180688C930E94FD1A0C9479
:1001F0001E0100919200003018F011F00C940201E1
:100200000C941E01A0E6B0E00E94E01C082F0E3006
:1002100010F00C941701A2E9B0E08C91A0E6B0E0D8
:100220008F930E94B71A8F918D9388278C93A2E9A0
:10023000B0E08C910E94001B0C941E01A0E9B0E07C
:100240008C9187FB0EF009C0E0E6F0E0A0E8B0E09A
:100250000E94B21A379A0C945C01A0E9B0E08C912C
:1002600085FB0EF425C0EFE9F0E0019111274FE086
:1002700050E00E94991AE1EFFFEFE00FF11FA0E8B4
:10028000B0E00E94D91CAFE9B0E08C918F5F8C93F5
:10029000E2ECF1E0BB27A4E10E94CF1C00919F009B
:1002A000041708F403C081E080939F000C945C0164
:1002B000A0E8B0E00E94511BA0E9B0E08C918F7ED5
:1002C0008C93A0E9B0E08C9187FB81E00EF080E098
:1002D0008F93A0E9B0E08C9185FB81E00EF480E083
:1002E0009F91892B882311F40C943904A0E9B0E084
:1002F0008C9186FB0EF45FC2A0E8B0E00E94E01C87
:10030000AEE1B1E08C93A0E1B1E0E4EFF9E30E944B
:10031000AC1A81E080931C0180E080931D01409124
:100320001E0100911C01041718F011F00C94B60383
:1003300080911C01E0E8F0E001E0A0E7B0E00E945D
:10034000BE1AA0E7B0E08C91A2E9B0E08C9381E402
:10035000482F00919200041781E008F480E08F9309
:100360008AE5482F00919200041781E010F009F00F
:1003700080E09F9189238F9381E6482F009192001E
:10038000041781E008F480E09F91892B8F938AE71E
:10039000482F00919200041781E010F009F080E0EE
:1003A0009F918923882311F40C94FB0180911C01F7
:1003B000E0E8F0E002E0A6E1B1E00E94BE1AACE1A4
:1003C000B1E08C918E5F8C9300911D01003011F093
:1003D0000C94F201E6E1F1E0A0E1B1E00E94B21A72
:1003E0000C94F901E6E1F1E0FA93EA930E94DB084C
:1003F00022960C94B40389E3482F009192000417CD
:1004000081E010F009F080E08F9380E3482F0091A5
:100410009200041781E008F480E09F9189238823EB
:1004200011F40C94640280E080931F01ACE1B1E010
:100430008C918F5F8C93AFE1B1E08C918F5F8C9347
:1004400080911C01E0E8F0E001E0A0E7B0E00E944C
:10045000BE1AA0E7B0E08C91A2E9B0E08C9389E3EA
:10046000482F00919200041781E010F009F080E01D
:100470008F9380E3482F00919200041781E008F4E5
:1004800080E09F918923882311F40C9449020C94F5
:10049000160200911C0140911F01041BA4E9B0E069
:1004A0000C9380919400E0E8F0E000911F01A6E138
:1004B000B1E00E94BE1AE6E1F1E0FA93EA930E94ED
:1004C000DB0822960C94B4038AE2482F0091920034
:1004D000041711F00C947E02ADE1B1E00D911127EB
:1004E00043E050E00E94991AA5EEB0E0A00FB11FC2
:1004F000E6EFF9E30E94AC1A0C94AF038BE2482FAD
:10050000041711F00C949602ADE1B1E00D911127A2
:1005100043E050E00E94991AA5EEB0E0A00FB11F91
:10052000E8EFF9E30E94AC1A0C94AF038DE3482F77
:10053000041711F00C94B10281E080931D01A4EE28
:10054000B0E00E94511BA8EEB0E0E8EFF9E30E9492
:10055000AC1AE6E1F1E0A0E1B1E00E94B21A0C941D
:10056000AF038AE3482F041711F00C94CC020E94C9
:10057000D406A7E9B0E00D911C91003050E01507BA
:1005800011F40C94CA02A0E9B0E08C9180618C93C4
:100590000C94B6030C94AF0381E2482F041711F0BA
:1005A0000C94E7020E94D406A7E9B0E00D911C91DB
:1005B000003050E0150711F00C94E502A0E9B0E01E
:1005C0008C9180618C930C94B6030C94AF038BE3F5
:1005D000482F041711F00C94FA020E94910CA0E12C
:1005E000B1E0E4EFF9E30E94AC1A80E080931D01D2
:1005F0000C94AF038DE2482F041711F00C941203F2
:10060000ADE1B1E00D91112743E050E00E94991A4D
:10061000A5EEB0E0A00FB11FEAEFF9E30E94AC1A1B
:100620000C94AF038FE2482F041711F00C942A03A7
:10063000ADE1B1E00D91112743E050E00E94991A1D
:10064000A5EEB0E0A00FB11FECEFF9E30E94AC1AE9
:100650000C94AF038CE5482F041711F00C9442035F
:10066000ADE1B1E00D91112743E050E00E94991AED
:10067000A5EEB0E0A00FB11FEEEFF9E30E94AC1AB7
:100680000C94AF038EE3482F041711F00C945A0317
:10069000ADE1B1E00D91112743E050E00E94991ABD
:1006A000A5EEB0E0A00FB11FE0E0FAE30E94AC1AA3
:1006B0000C94AF038CE3482F041711F00C947203D1
:1006C000ADE1B1E00D91112743E050E00E94991A8D
:1006D000A5EEB0E0A00FB11FE2E0FAE30E94AC1A71
:1006E0000C94AF038BE5482F041711F00C9487038B
:1006F00082E080931D01A6EEB0E00E94511BABEE9C
:10070000B0E0E8EFF9E30E94AC1A0C94AF038DE57A
:10071000482F041711F00C949F0381E080931D0172
:10072000A0E7B0E0E4E0FAE30E94AC1AE0E7F0E012
:10073000FA93EA930E94DB0822960C94AF0380E2BE
:10074000482F041711F00C94A7030C94AF0385E213
:10075000482F041711F00C94AF030C94B603ACE1CE
:10076000B1E08C918F5F8C930C948F010E94850C6B
:10077000A0E9B0E08C9184FB0EF402C00E94910CC1
:10078000A0E9B0E08C9186FB81E00EF480E08F93CD
:10079000A0E9B0E08C9185FB81E00EF080E09F91B4
:1007A0008923882311F40C94D903E0E0FAE30E9432
:1007B000F61A0C94280481E10E94331BE0E6F0E075
:1007C000A881B98102E00E94C41AA881B981E6E03B
:1007D000FAE30E94E61C0FB681E1481A8827580AFE
:1007E00022960FBE11F00C940604E2ECF1E0AFE9A2
:1007F000B0E00E94BC1CA0E9B0E08C918F7B8C9390
:10080000E0E0FAE30E94F61A0C942804E0E6F0E037
:10081000A0E7B0E00EE00E94C41A00919F000F31E3
:1008200010F00C942804EFE9F0E0019111274FE05B
:1008300050E00E94991AE1EFFFEFE00FF11FA0E7EF
:10084000B0E00E94C71CAFE9B0E08C918F5F8C9341
:10085000A0E9B0E08C9187FB0EF004C0A0E6B0E008
:100860000E94511BA0E9B0E08C918F778C930C947F
:100870003F04379885B78F70806485BF88950C9446
:10088000C3000F921F922F923F924F925F926F92EE
:100890007F928F929F92AF92BF920F931F932F934D
:1008A0003F934F935F936F937F938F939F93AF93F8
:1008B000BF93CF93DF93EF93FF938FB78F93A0E90D
:1008C000B0E08C9185FB0EF4A1C181E080930F0113
:1008D00000910F010A3018F011F00C949504AFE06C
:1008E000B1E0AD90BB24AEECB0E0AA0CBB1CAA0DED
:1008F000BB1D0D911C91003050E0150711F40C94B4
:100900008D04AFE0B1E0AD90BB24AEECB0E0AA0C3A
:10091000BB1CAA0DBB1D0E94541AAFE0B1E08C9124
:100920008F5F8C9311F00C946804AEE0B1E0AD9051
:10093000BB24AAEFB0E0AA0CBB1CAA0DBB1D8D9175
:100940009C91A9E9B0E08D939C93AEE0B1E0AD90AD
:10095000BB24AEEFB0E0AA0CBB1CAA0DBB1D8D9151
:100960009C91ABE9B0E08D939C93ABE9B0E00D9125
:100970001C91A9E9B0E04D915C91041B150BABE90A
:10098000B0E00D931C93ABE9B0E00D911C91063AD9
:1009900050E015071CF011F00C94D0040C94D8040E
:1009A00086EA90E0ABE9B0E08D939C930C94E90467
:1009B000ABE9B0E00D911C910A355FEF15070CF41F
:1009C00002C00C94E9048AE59FEFABE9B0E08D9397
:1009D0009C93AEE0B1E0AD90BB24AEEEB0E0AA0CCB
:1009E000BB1CAA0DBB1D8D919C91ADE9B0E08D9310
:1009F0009C93ABE9B0E00D911C91ADE9B0E04D9155
:100A00005C910E945A1AA9E9B0E00D931C930E94D0
:100A1000B408A9E9B0E08D919C91AEE0B1E0AD9051
:100A2000BB24A2E0B1E0AA0CBB1CAA0DBB1D8D9398
:100A30009C93AEE0B1E0AD90BB24A2EFB0E0AA0C75
:100A4000BB1CAA0DBB1D8D919C91ADE9B0E08D93AF
:100A50009C93ADE9B0E00D911C91ABE9B0E04D91F4
:100A60005C910E945A1AA9E9B0E00D931C93A9E980
:100A7000B0E00D911C9140E150E00E945F1AA9E99D
:100A8000B0E04D935C93AEE0B1E0AD90BB24A2EF3B
:100A9000B0E0AA0CBB1CAA0DBB1D0D911C9100302F
:100AA00050E0150711F00C946105AEE0B1E0AD9097
:100AB000BB24A6E0B1E0AA0CBB1CAA0DBB1D0E9482
:100AC000511BAEE0B1E0AD90BB24A6E0B1E0AA0CB2
:100AD000BB1CAA0DBB1D8D919C91ADE9B0E08D931F
:100AE0009C93ADE9B0E00D911C91A9E9B0E04D9166
:100AF0005C91040F151FA9E9B0E00D931C930E94AF
:100B0000B408A9E9B0E08D919C91AEE0B1E0AD9060
:100B1000BB24A6E0B1E0AA0CBB1CAA0DBB1D8D93A3
:100B20009C93AEE0B1E0AD90BB24A2E0B1E0AA0C92
:100B3000BB1CAA0DBB1D8D919C91ADE9B0E08D93BE
:100B40009C93ADE9B0E00D911C91A9E9B0E04D9105
:100B50005C91040F151FA9E9B0E00D931C930E944E
:100B6000B408A9E9B0E00D911C9140E150E00E9469
:100B70005F1AA9E9B0E04D935C93A9E9B0E00D914B
:100B80001C91003050E015070CF402C00C94CC0509
:100B9000A9E9B0E00E94511BA9E9B0E08D919C91B8
:100BA000AEE0B1E0AD90BB24A2E0B1E0AA0CBB1C6A
:100BB000AA0DBB1D8D939C9300910E01013011F085
:100BC0000C94030680E080930E010FEF13E0A2E087
:100BD000B1E04D915C91041B150BBB27A0E18D91F9
:100BE0009C919BBD8ABD0FEF13E0A4E0B1E04D9155
:100BF0005C91041B150BBB27A0E18D919C9199BDC5
:100C000088BD0C94060681E080930E018F918FBF02
:100C1000FF91EF91DF91CF91BF91AF919F918F9114
:100C20007F916F915F914F913F912F911F910F9104
:100C3000BF90AF909F908F907F906F905F904F90FC
:100C40003F902F901F900F9018950E944A15A881F1
:100C5000B9818C9187528C93E881F981A190BB2452
:100C6000E2ECF1E0AA0CBB1CEA0DFB1DBB27A0E1E6
:100C70000E94D11C003050E015070CF402C00C9407
:100C80005106E881F981A190BB24E2ECF1E0AA0CC5
:100C9000BB1CEA0DFB1D00E010E0A0E1BB270E9499
:100CA000BE1CA0E9B0E08C9183FB0EF43FC0A8818C
:100CB000B981AD90BB24AAEBB0E0AA0CBB1CAA0D75
:100CC000BB1D0D911C91E881F981A190BB24E2EC40
:100CD000F1E0AA0CBB1CEA0DFB1DBB27A4E10E949E
:100CE000D11C040F151FA7E9B0E00D931C93A7E9D1
:100CF000B0E04D915C91A881B981AD90BB24A6EA8A
:100D0000B0E0AA0CBB1CAA0DBB1D0D911C910417D1
:100D100015071CF011F00C948F060C949406A0E9B2
:100D2000B0E08C9188608C930C94D106A881B98135
:100D3000AD90BB24AAEBB0E0AA0CBB1CAA0DBB1D56
:100D40000D911C91E881F981A190BB24E2ECF1E0C6
:100D5000AA0CBB1CEA0DFB1DBB27A4E10E94D11C01
:100D6000041B150BA7E9B0E00D931C93A7E9B0E0B5
:100D70004D915C91A881B981AD90BB24A6EAB0E009
:100D8000AA0CBB1CAA0DBB1D0D911C9104171507C5
:100D90000CF402C00C94D106A0E9B0E08C91877FDE
:100DA0008C930E94A61808950E94640C82E6482F36
:100DB00000919200041711F00C94F20680919300B8
:100DC0008A95809393000E944A15A0E9B0E08C9127
:100DD00083FBA7E9B0E0882780F98D9388278C935F
:100DE0000C94B30882E4482F041711F00C941007F8
:100DF000809193008A95809393000E944A15A0E900
:100E0000B0E08C9183FB882780F9809580FBA7E96F
:100E1000B0E0882780F98D9388278C930C94B308D1
:100E200089E6482F041711F00C942A07A3E9B0E0D3
:100E30008C91875F8C930E944A15A0E9B0E08C9159
:100E400083FBA7E9B0E0882780F98D9388278C93EE
:100E50000C94B30889E4482F041711F00C94480748
:100E6000A3E9B0E08C91875F8C930E944A15A0E9BA
:100E7000B0E08C9183FB882780F9809580FBA7E9FF
:100E8000B0E0882780F98D9388278C930C94B30861
:100E90008FE6482F041711F00C946207A3E9B0E025
:100EA0008C918D5E8C930E944A15A0E9B0E08C91E4
:100EB00083FBA7E9B0E0882780F98D9388278C937E
:100EC0000C94B3088FE4482F041711F00C9480079A
:100ED000A3E9B0E08C918D5E8C930E944A15A0E945
:100EE000B0E08C9183FB882780F9809580FBA7E98F
:100EF000B0E0882780F98D9388278C930C94B308F1
:100F000084E6482F041711F00C949A07A3E9B0E087
:100F10008C91835E8C930E944A15A0E9B0E08C917D
:100F200083FBA7E9B0E0882780F98D9388278C930D
:100F30000C94B30888E6482F041711F00C94C207EC
:100F4000A3E9B0E08C91895D8C935A924A9280918A
:100F50009300A42DB52D8C9381E00E94501A0E941D
:100F60002506229681E00E944C1AA0E9B0E08C91FF
:100F700083FBA7E9B0E0882780F98D9388278C93BD
:100F80000C94B30888E4482F041711F00C94EE0772
:100F9000A3E9B0E08C91895D8C935A924A9280913A
:100FA0009300A42DB52D8C9381E00E94501A0E94CD
:100FB0002506229681E00E944C1AA0E9B0E08C91AF
:100FC00083FB882780F9809580FBA7E9B0E088271C
:100FD00080F98D9388278C930C94B30882E7482F6F
:100FE000041711F00C940608A3E9B0E0AD90BB24FF
:100FF000A6EAB0E0AA0CBB1CAA0DBB1D8D919C916A
:10100000A7E9B0E08D939C930C94B30883E7482F35
:10101000041711F00C941E08A3E9B0E0AD90BB24B6
:10102000AAEBB0E0AA0CBB1CAA0DBB1D8D919C9134
:10103000A7E9B0E08D939C930C94B30880E7482F08
:10104000041711F00C943808F894A3E9B0E0AD90BF
:10105000BB24ACEEB0E0AA0CBB1CAA0DBB1D8D914D
:101060009C91A7E9B0E08D939C9378940C94B3087D
:1010700085E7482F041711F00C946F080091930036
:10108000093010F00C945608A3E9B0E08C9181501F
:101090008C93A3E9B0E08C91806C87B90E942A1BE5
:1010A000A7E9B0E08D939C930C946D08A3E9B0E0A0
:1010B0008C918E5F8C93F894A3E9B0E0AD90BB2443
:1010C000ACEEB0E0AA0CBB1CAA0DBB1D8D919C918F
:1010D000A7E9B0E08D939C9378940C94B30884E7CF
:1010E000482F041711F00C948908F894A3E9B0E094
:1010F000AD90BB24AEECB0E0AA0CBB1CAA0DBB1D8E
:101100008D919C91A7E9B0E08D939C9378940C9479
:10111000B30885E6482F041711F00C949F08E3E903
:10112000F0E0A190BB24E2ECF1E0AA0CBB1CEA0DBC
:10113000FB1DA7E9B0E00E94D11C0C94B30886E621
:10114000482F041711F00C94B308E3E9F0E0A190E4
:10115000BB24E6EDF1E0AA0CBB1CEA0DFB1DA7E9E0
:10116000B0E00E94D11C0895A9E9B0E00D911C9156
:10117000013050EC15070CF402C00C94C70881E054
:1011800090ECA9E9B0E08D939C930C94DA08A9E95E
:10119000B0E00D911C910F3F5FE315071CF011F0BB
:1011A0000C94D4080C94DA088FEF9FE3A9E9B0E01F
:1011B0008D939C930895A881B9818C91A2E9B0E0A8
:1011C0008C9389E3482F00919200041781E010F07E
:1011D00009F080E08F9380E3482F0091920004177C
:1011E00081E008F480E09F918923882311F40C9416
:1011F0000309A881B9810E94891CA7E9B0E00D9379
:101200001C930C941F0B8DE5482F0091920004173E
:1012100011F00C94240900911D0141E0040FA3E991
:10122000B0E00C93A3E9B0E0AD90BB24A2EEB0E037
:10123000AA0CBB1CAA0DBB1D8D919C91A7E9B0E027
:101240008D939C930C941F0B82E0E881F98101E05F
:10125000A0E7B0E00E94BE1AA0E7B0E00E94891C9F
:10126000A3E9B0E00C9382E7482F009192000417A5
:1012700011F00C945209A3E9B0E08C918F5F8C932C
:10128000A3E9B0E0AD90BB24A6EAB0E0AA0CBB1C79
:10129000AA0DBB1D8D919C91A7E9B0E08D939C9305
:1012A0000C941F0B83E7482F041711F00C946F095F
:1012B000A3E9B0E08C918F5F8C93A3E9B0E0AD908F
:1012C000BB24AAEBB0E0AA0CBB1CAA0DBB1D8D91E0
:1012D0009C91A7E9B0E08D939C930C941F0B80E741
:1012E000482F041711F00C948E09A3E9B0E08C91FB
:1012F0008F5F8C93F894A3E9B0E0AD90BB24ACEE83
:10130000B0E0AA0CBB1CAA0DBB1D8D919C91A7E956
:10131000B0E08D939C9378940C941F0B85E7482F35
:10132000041711F00C94C00900919300083010F0DC
:101330000C94A709A3E9B0E08C91806C87B90E9456
:101340002A1BA7E9B0E08D939C930C94BE09A3E9F6
:10135000B0E08C918D5F8C93F894A3E9B0E0AD90F0
:10136000BB24ACEEB0E0AA0CBB1CAA0DBB1D8D913A
:101370009C91A7E9B0E08D939C9378940C941F0BFB
:1013800084E7482F041711F00C94DF09A3E9B0E0BB
:101390008C918F5F8C93F894A3E9B0E0AD90BB245F
:1013A000AEECB0E0AA0CBB1CAA0DBB1D8D919C91AC
:1013B000A7E9B0E08D939C9378940C941F0B85E67D
:1013C000482F041711F00C94FA09A3E9B0E08C91AE
:1013D0008F5F8C93E3E9F0E0A190BB24E2ECF1E0B5
:1013E000AA0CBB1CEA0DFB1DA7E9B0E00E94D11CB2
:1013F0000C941F0B86E6482F041711F00C94150A65
:10140000A3E9B0E08C918F5F8C93E3E9F0E0A190C9
:10141000BB24E6EDF1E0AA0CBB1CEA0DFB1DA7E91D
:10142000B0E00E94D11C0C941F0B82E6482F0417D9
:1014300011F00C942A0A0E944A15A0E9B0E08C91A0
:1014400083FBA7E9B0E0882780F98D9388278C93E8
:101450000C941F0B82E4482F041711F00C94430ADC
:101460000E944A15A0E9B0E08C9183FB882780F99F
:10147000809580FBA7E9B0E0882780F98D938827C5
:101480008C930C941F0B89E6482F041711F00C94D1
:101490005D0AA3E9B0E08C91865F8C930E944A15A7
:1014A000A0E9B0E08C9183FBA7E9B0E0882780F940
:1014B0008D9388278C930C941F0B89E4482F041775
:1014C00011F00C947B0AA3E9B0E08C91865F8C93B9
:1014D0000E944A15A0E9B0E08C9183FB882780F92F
:1014E000809580FBA7E9B0E0882780F98D93882755
:1014F0008C930C941F0B8FE6482F041711F00C945B
:10150000950AA3E9B0E08C918C5E8C930E944A15F9
:10151000A0E9B0E08C9183FBA7E9B0E0882780F9CF
:101520008D9388278C930C941F0B8FE4482F0417FE
:1015300011F00C94B30AA3E9B0E08C918C5E8C930B
:101540000E944A15A0E9B0E08C9183FB882780F9BE
:10155000809580FBA7E9B0E0882780F98D938827E4
:101560008C930C941F0B84E6482F041711F00C94F5
:10157000CD0AA3E9B0E08C91825E8C930E944A155B
:10158000A0E9B0E08C9183FBA7E9B0E0882780F95F
:101590008D9388278C930C941F0B88E6482F041793
:1015A00011F00C94F50AA3E9B0E08C91885D8C935E
:1015B0005A924A9280919300A42DB52D8C9381E08C
:1015C0000E94501A0E942506229681E00E944C1A21
:1015D000A0E9B0E08C9183FBA7E9B0E0882780F90F
:1015E0008D9388278C930C941F0B88E4482F041745
:1015F00011F00C941F0BA3E9B0E08C91885D8C93E3
:101600005A924A9280919300A42DB52D8C9381E03B
:101610000E94501A0E942506229681E00E944C1AD0
:10162000A0E9B0E08C9183FB882780F9809580FB4E
:10163000A7E9B0E0882780F98D9388278C93ADE1E6
:10164000B1E00D91112743E050E00E94991AA5EEF8
:10165000B0E0A00FB11F8C91A2E9B0E08C938AE2B8
:10166000482F00919200041711F00C94570BADE134
:10167000B1E0AD90BB24A2EEB0E0AA0CBB1CAA0D59
:10168000BB1D0D911C91A7E9B0E04D915C910E94AA
:101690005A1AADE1B1E0AD90BB24A2EEB0E0AA0CC5
:1016A000BB1CAA0DBB1D0D931C930C94630C8BE209
:1016B000482F041711F00C947D0BADE1B1E0AD9013
:1016C000BB24A2EEB0E0AA0CBB1CAA0DBB1D0D9161
:1016D0001C91A7E9B0E04D915C91040F151FADE19D
:1016E000B1E0AD90BB24A2EEB0E0AA0CBB1CAA0DE9
:1016F000BB1D0D931C930C94630C8DE2482F0417B3
:1017000011F00C94A30BADE1B1E0AD90BB24A2EEBF
:10171000B0E0AA0CBB1CAA0DBB1D0D911C91A7E942
:10172000B0E04D915C91041B150BADE1B1E0AD90C3
:10173000BB24A2EEB0E0AA0CBB1CAA0DBB1D0D93EE
:101740001C930C94630C8FE2482F041711F00C9437
:10175000C90BADE1B1E0AD90BB24A2EEB0E0AA0CA4
:10176000BB1CAA0DBB1D0D911C91A7E9B0E04D91CA
:101770005C910E945F1AADE1B1E0AD90BB24A2EE96
:10178000B0E0AA0CBB1CAA0DBB1D4D935C930C943E
:10179000630C8CE5482F041711F00C94EF0BADE1AE
:1017A000B1E0AD90BB24A2EEB0E0AA0CBB1CAA0D28
:1017B000BB1D0D911C91A7E9B0E04D915C910E9479
:1017C0005F1AADE1B1E0AD90BB24A2EEB0E0AA0C8F
:1017D000BB1CAA0DBB1D0D931C930C94630C8EE3D4
:1017E000482F041711F00C942B0CA7E9B0E04D9191
:1017F0005C91ADE1B1E0AD90BB24A2EEB0E0AA0CEB
:10180000BB1CAA0DBB1D0D911C91041715071CF0E4
:1018100011F00C940D0C0C941D0C81E090E0ADE1E6
:10182000B1E0AD90BB24A2EEB0E0AA0CBB1CAA0DA7
:10183000BB1D8D939C930C94290CADE1B1E0AD9050
:10184000BB24A2EEB0E0AA0CBB1CAA0DBB1D0E94DB
:10185000511B0C94630C8CE3482F041711F00C946B
:10186000630CA7E9B0E04D915C91ADE1B1E0AD90C2
:10187000BB24A2EEB0E0AA0CBB1CAA0DBB1D0D91AF
:101880001C91041715070CF402C00C94570C81E04E
:1018900090E0ADE1B1E0AD90BB24A2EEB0E0AA0CC7
:1018A000BB1CAA0DBB1D8D939C930C94630CADE1E6
:1018B000B1E0AD90BB24A2EEB0E0AA0CBB1CAA0D17
:1018C000BB1D0E94511B089581E0E0E1F1E001E0C1
:1018D000A0E7B0E00E94BE1AA0E7B0E08C91A2E9B8
:1018E000B0E08C9382E0E0E1F1E001E0A0E7B0E05D
:1018F0000E94BE1AA0E7B0E00E94891C002F41E0C0
:10190000040FA3E9B0E00C93089500915301053052
:1019100018F011F00C948E0C0C94900C0C94850C17
:1019200008950E94640C82E7482F009192000417EA
:1019300011F00C94E80C00911D01003011F00C9492
:10194000CE0C0091930041E0041BA4E9B0E00C939D
:101950000E94850CEAE0FAE30E94F61AA0EFB3E0D9
:10196000E4E9F0E00E94451C0E94EE1AECE0FAE384
:101970000E94F61AA0EFB3E0E3E9F0E0A190BB24E7
:10198000E6EAF0E0AA0CBB1CEA0DFB1D0E943E1C1F
:101990000E94EE1A0E94FD1A0C94E60CADE1B1E033
:1019A000AD90BB24A2EEB0E0AA0CBB1CAA0DBB1DDF
:1019B0008D919C91A3E9B0E0AD90BB24A6EAB0E084
:1019C000AA0CBB1CAA0DBB1D8D939C930C944915AE
:1019D00083E7482F041711F00C943B0D00911D0173
:1019E000003011F00C94210D0091930041E0041B94
:1019F000A4E9B0E00C930E94850CEEE0FAE30E94AB
:101A0000F61AA0EFB3E0E4E9F0E00E94451C0E9462
:101A1000EE1AECE0FAE30E94F61AA0EFB3E0E3E975
:101A2000F0E0A190BB24EAEBF0E0AA0CBB1CEA0DAD
:101A3000FB1D0E943E1C0E94EE1A0E94FD1A0C948F
:101A4000390DADE1B1E0AD90BB24A2EEB0E0AA0C3F
:101A5000BB1CAA0DBB1D8D919C91A3E9B0E0AD907C
:101A6000BB24AAEBB0E0AA0CBB1CAA0DBB1D8D9336
:101A70009C930C94491580E7482F041711F00C949F
:101A8000AE0D00911D01003011F00C94760D009107
:101A9000930041E0041BA4E9B0E00C930E94850C84
:101AA000F894E0E1FAE30E94F61AA0EFB3E0E4E96B
:101AB000F0E00E94451C0E94EE1AECE0FAE30E945E
:101AC000F61AA0EFB3E0E3E9F0E0A190BB24ECEE5E
:101AD000F0E0AA0CBB1CEA0DFB1D0E943E1C0E94FC
:101AE000EE1A0E94FD1A78940C94AC0DF894ADE1B6
:101AF000B1E0AD90BB24A2EEB0E0AA0CBB1CAA0DD5
:101B0000BB1D8D919C91A3E9B0E0AD90BB24ACEEE0
:101B1000B0E0AA0CBB1CAA0DBB1D8D939C93009139
:101B20009300063010F009F016C0E3E9F0E0A19050
:101B3000BB24EAEEF1E0AA0CBB1CEA0DFB1DA3E9F5
:101B4000B0E0AD90BB24ACEEB0E0AA0CBB1CAA0D7B
:101B5000BB1D0E94BE1C78940C94491585E7482F44
:101B6000041711F00C94200E00911D01003011F0AB
:101B70000C941E0E00919300093010F00C94EC0DA3
:101B8000809193008A95809393000E94850CE2E1F6
:101B9000FAE30E94F61AA0EFB3E0E3E9F0E00E9456
:101BA000451C0E94EE1AECE0FAE30E94F61AA3E943
:101BB000B0E08C91806C87B90E942A1B082F192FE6
:101BC000A0EFB3E0FF27E0E10E94361C0E94EE1A6E
:101BD0000E94FD1A0C941E0EA3E9B0E08C918E5F5A
:101BE0008C930091930043E0041BA4E9B0E00C93B4
:101BF0000E94850CF894E2E1FAE30E94F61AA0EF45
:101C0000B3E0E4E9F0E00E94451C0E94EE1AECE02B
:101C1000FAE30E94F61AA0EFB3E0E3E9F0E0A19046
:101C2000BB24ECEEF0E0AA0CBB1CEA0DFB1D0E94ED
:101C30003E1C0E94EE1A0E94FD1A78940C944915DD
:101C400084E7482F041711F00C94770E00911D01C2
:101C5000003011F00C945B0E0091930041E0041BE6
:101C6000A4E9B0E00C930E94850CF894E4E1FAE357
:101C70000E94F61AA0EFB3E0E4E9F0E00E94451CF0
:101C80000E94EE1AECE0FAE30E94F61AA0EFB3E02D
:101C9000E3E9F0E0A190BB24EEECF0E0AA0CBB1C61
:101CA000EA0DFB1D0E943E1C0E94EE1A0E94FD1AC6
:101CB00078940C94750EF894ADE1B1E0AD90BB242E
:101CC000A2EEB0E0AA0CBB1CAA0DBB1D8D919C918D
:101CD000A3E9B0E0AD90BB24AEECB0E0AA0CBB1C15
:101CE000AA0DBB1D8D939C9378940C94491585E6A1
:101CF000482F041711F00C94CE0E00911D010030F6
:101D000011F00C94B60E0091930041E0041BA4E97D
:101D1000B0E00C930E94850CE3E9F0E0A190BB24B5
:101D2000E2ECF1E0AA0CBB1CEA0DFB1DA5E9B0E05A
:101D30000E94D11CE6E1FAE30E94F61AA0EFB3E09C
:101D4000E4E9F0E00E94451C0E94EE1AECE0FAE3A0
:101D50000E94F61AA0EFB3E0E5E9F0E00E943E1C15
:101D60000E94EE1A0E94FD1A0C94CC0EE3E9F0E0FA
:101D7000A190BB24E2ECF1E0AA0CBB1CEA0DFB1D18
:101D8000ADE1B1E0AD90BB24A2EEB0E0AA0CBB1C6B
:101D9000AA0DBB1D0E94BE1C0C94491586E6482F57
:101DA000041711F00C94250F00911D01003011F063
:101DB0000C940D0F0091930041E0041BA4E9B0E0E6
:101DC0000C930E94850CE3E9F0E0A190BB24E6EDC2
:101DD000F1E0AA0CBB1CEA0DFB1DA5E9B0E00E94D6
:101DE000D11CE8E1FAE30E94F61AA0EFB3E0E4E9BF
:101DF000F0E00E94451C0E94EE1AECE0FAE30E941B
:101E0000F61AA0EFB3E0E5E9F0E00E943E1C0E9464
:101E1000EE1A0E94FD1A0C94230FE3E9F0E0A19062
:101E2000BB24E6EDF1E0AA0CBB1CEA0DFB1DADE105
:101E3000B1E0AD90BB24A2EEB0E0AA0CBB1CAA0D91
:101E4000BB1D0E94BE1C0C94491582E6482F041746
:101E500011F00C947D0F809193008A9580939300EC
:101E600000911D01003011F00C945B0F0E94850C55
:101E70000E944A15EAE1FAE30E94F61AA0EFB3E0E5
:101E8000E3E9F0E00E94451C0E94EE1AECE0FAE360
:101E90000E94F61AA0E9B0E08C9183FBA0EFB3E0BA
:101EA0000E94591B8D9388278C930E94EE1A0E94E2
:101EB000FD1A0C947B0FADE1B1E0AD90BB24A2EE16
:101EC000B0E0AA0CBB1CAA0DBB1D0D911C910030EB
:101ED00050E0150711F00C94740FA0E9B0E08C915C
:101EE000877F8C930C94790FA0E9B0E08C91886087
:101EF0008C930E94A6180C94491582E4482F04176D
:101F000011F00C94E20F809193008A9580939300D6
:101F100000911D01003011F00C94C00F0E944A1571
:101F2000A0E9B0E08C9183FB882780F9809580FB45
:101F3000A0E9B0E08C9183F98C930E94850CECE1D0
:101F4000FAE30E94F61AA0EFB3E0E3E9F0E00E94A2
:101F5000451C0E94EE1AECE0FAE30E94F61AA0E992
:101F6000B0E08C9183FBA0EFB3E00E94591B8D93EE
:101F700088278C930E94EE1A0E94FD1A0C94E00FA1
:101F8000ADE1B1E0AD90BB24A2EEB0E0AA0CBB1C69
:101F9000AA0DBB1D0D911C91003050E0150711F0EA
:101FA0000C94D90FA0E9B0E08C9188608C930C94CC
:101FB000DE0FA0E9B0E08C91877F8C930E94A61879
:101FC0000C94491589E6482F041711F00C941F1042
:101FD000A3E9B0E08C91875F8C93009193004AE075
:101FE000041BA4E9B0E00C9300911D01003011F036
:101FF0000C941D100E944A150E94850CEEE1FAE334
:102000000E94F61AA0EFB3E0E4E9F0E00E94451C5C
:102010000E94EE1AECE0FAE30E94F61AA0E9B0E0A2
:102020008C9183FBA0EFB3E00E94591B8D9388270E
:102030008C930E94EE1A0E94FD1A0C94491589E4B3
:10204000482F041711F00C946910A3E9B0E08C91AB
:10205000875F8C93009193004AE0041BA4E9B0E0F1
:102060000C9300911D01003011F00C9467100E9438
:102070004A15A0E9B0E08C9183FB882780F9809510
:1020800080FBA0E9B0E08C9183F98C930E94850CD1
:10209000E0E2FAE30E94F61AA0EFB3E0E3E9F0E031
:1020A0000E94451C0E94EE1AECE0FAE30E94F61A28
:1020B000A0E9B0E08C9183FBA0EFB3E00E94591B34
:1020C0008D9388278C930E94EE1A0E94FD1A0C941F
:1020D00049158FE6482F041711F00C94C810A3E996
:1020E000B0E08C918D5E8C930091930044E1041BD1
:1020F000A4E9B0E00C9300911D01003011F00C94A4
:10210000A6100E944A150E94850CE2E2FAE30E94A2
:10211000F61AA0EFB3E0E4E9F0E00E94451C0E944B
:10212000EE1AECE0FAE30E94F61AA0E9B0E08C9116
:1021300083FBA0EFB3E00E94591B8D9388278C93FB
:102140000E94EE1A0E94FD1A0C94C610ADE1B1E097
:10215000AD90BB24A2EEB0E0AA0CBB1CAA0DBB1D27
:102160000D911C91003050E0150711F00C94BF1038
:10217000A0E9B0E08C91877F8C930C94C410A0E907
:10218000B0E08C9188608C930E94A6180C9449153D
:102190008FE4482F041711F00C943411A3E9B0E038
:1021A0008C918D5E8C930091930044E1041BA4E913
:1021B000B0E00C9300911D01003011F00C9412114D
:1021C0000E944A15A0E9B0E08C9183FB882780F932
:1021D000809580FBA0E9B0E08C9183F98C930E94FC
:1021E000850CE4E2FAE30E94F61AA0EFB3E0E4E91A
:1021F000F0E00E94451C0E94EE1AECE0FAE30E9417
:10220000F61AA0E9B0E08C9183FBA0EFB3E00E9446
:10221000591B8D9388278C930E94EE1A0E94FD1AF9
:102220000C943211ADE1B1E0AD90BB24A2EEB0E070
:10223000AA0CBB1CAA0DBB1D0D911C91003050E0D7
:10224000150711F00C942B11A0E9B0E08C91886077
:102250008C930C943011A0E9B0E08C91877F8C9323
:102260000E94A6180C94491584E6482F041711F013
:102270000C947111A3E9B0E08C91835E8C93009172
:1022800093004EE1041BA4E9B0E00C9300911D0102
:10229000003011F00C946F110E944A150E94850CB9
:1022A000E6E2FAE30E94F61AA0EFB3E0E4E9F0E018
:1022B0000E94451C0E94EE1AECE0FAE30E94F61A16
:1022C000A0E9B0E08C9183FBA0EFB3E00E94591B22
:1022D0008D9388278C930E94EE1A0E94FD1A0C940D
:1022E000491588E6482F041711F00C94BC11A3E996
:1022F000B0E08C91895D8C9300911D01003011F04C
:102300000C94BA115A924A9280919300A42DB52D43
:102310008C9381E00E94501A0E942506229681E04B
:102320000E944C1A0091930048E2041BA4E9B0E01B
:102330000C930E94850CE8E2FAE30E94F61AA0EFE3
:10234000B3E0E4E9F0E00E94451C0E94EE1AECE0E4
:10235000FAE30E94F61AA0E9B0E08C9183FBA0EFAB
:10236000B3E00E94591B8D9388278C930E94EE1A2C
:102370000E94FD1A0C94491588E4482F041711F0A7
:102380000C941412A3E9B0E08C91895D8C930091B8
:102390001D01003011F00C9412125A924A92809151
:1023A0009300A42DB52D8C9381E00E94501A0E94B9
:1023B0002506229681E00E944C1AA0E9B0E08C919B
:1023C00083FB882780F9809580FBA0E9B0E08C91A1
:1023D00083F98C930091930048E2041BA4E9B0E0D8
:1023E0000C930E94850CEAE2FAE30E94F61AA0EF31
:1023F000B3E0E4E9F0E00E94451C0E94EE1AECE034
:10240000FAE30E94F61AA0E9B0E08C9183FBA0EFFA
:10241000B3E00E94591B8D9388278C930E94EE1A7B
:102420000E94FD1A0C94491583E6482F041711F0F9
:102430000C94491500911D01003011F00C942012EC
:1024400000919300013011F00C9444120E94850C0D
:10245000ECE2FAE30E94F61A0E94FD1AECE3FAE3BA
:102460000E94F61A0E94FD1A0E94850CECE4FAE321
:102470000E94F61A0E94FD1AECE5FAE30E94F61A91
:102480000E94FD1A0C944915023011F00C94571259
:10249000A0E9B0E08C9180648C9381E080939F00F0
:1024A000A0E9B0E08C9180628C930C9449150330C4
:1024B00011F00C946212A0E9B0E08C9180628C93D0
:1024C0000C944915043011F00C947512A0E9B0E099
:1024D0008C918F7D8C93A0E9B0E08C918F7B8C9355
:1024E00081E080939F000C944915053011F00C9405
:1024F000CD12E2ECF1E0BB27A0E10E94CF1C0F3F20
:1025000081E009F480E08F93E2ECF1E0BB27A0E1E9
:102510000E94CF1C003081E009F480E09F91892364
:10252000882311F40C94CB12E2ECF1E0BB27A0E17C
:102530000E94CF1C41E0041BA4E9B0E00C9381E0B1
:10254000809393004091940000919300041718F039
:1025500011F00C94CB12E3E9F0E0019111274FE068
:1025600050E00E94991AE1EFFFEFE00FF11FA0E7A2
:10257000B0E00E94D91C0E94850CA0E7B0E00E9448
:10258000F01A0E94FD1AA3E9B0E08C918F5F8C9342
:1025900011F00C94A2120C944915063011F00C9411
:1025A00011150E94850CECE6FAE30E94F61A81E010
:1025B00080939300009193000A3018F011F00C946E
:1025C000FF120E94850CA0EFB3E0E3E9F0E0A190D8
:1025D000BB24E6EAF0E0AA0CBB1CEA0DFB1D0E943E
:1025E0003E1C0E94EE1AE0E7FAE30E94F61AA3E905
:1025F000B0E08C918F5F8C9311F00C94DA120E94F2
:10260000FD1AE2E7FAE30E94F61A81E08093930054
:10261000009193000A3018F011F00C942D130E94D1
:10262000850CA0EFB3E0E3E9F0E0A190BB24EAEB76
:10263000F0E0AA0CBB1CEA0DFB1D0E943E1C0E9490
:10264000EE1AE0E7FAE30E94F61AA3E9B0E08C91F3
:102650008F5F8C9311F00C9408130E94FD1AE6E72B
:10266000FAE30E94F61A81E08093930000919300B0
:102670000A3018F011F00C9461130E94850CE3E904
:10268000F0E0A190BB24E2ECF1E0AA0CBB1CEA0D47
:10269000FB1DA5E9B0E00E94D11CA0EFB3E0E5E985
:1026A000F0E00E943E1C0E94EE1AE0E7FAE30E946E
:1026B000F61AA3E9B0E08C918F5F8C9311F00C9423
:1026C00036130E94FD1AEAE7FAE30E94F61A81E047
:1026D00080939300009193000A3018F011F00C944D
:1026E00095130E94850CE3E9F0E0A190BB24E6ED90
:1026F000F1E0AA0CBB1CEA0DFB1DA5E9B0E00E94AD
:10270000D11CA0EFB3E0E5E9F0E00E943E1C0E947E
:10271000EE1AE0E7FAE30E94F61AA3E9B0E08C9122
:102720008F5F8C9311F00C946A130E94FD1AEEE7F0
:10273000FAE30E94F61A81E08093930000919300DF
:102740000A3018F011F00C94C5130E94850CF8940F
:10275000A0EFB3E0E3E9F0E0A190BB24EEECF0E001
:10276000AA0CBB1CEA0DFB1D0E943E1C0E94EE1A27
:10277000E0E7FAE30E94F61A7894A3E9B0E08C91BE
:102780008F5F8C9311F00C949E130E94FD1AE2E867
:10279000FAE30E94F61A81E080939300009193007F
:1027A0000A3018F011F00C94F5130E94850CF8947F
:1027B000A0EFB3E0E3E9F0E0A190BB24ECEEF0E0A1
:1027C000AA0CBB1CEA0DFB1D0E943E1C0E94EE1AC7
:1027D000E0E7FAE30E94F61A7894A3E9B0E08C915E
:1027E0008F5F8C9311F00C94CE130E94FD1AE6E8D3
:1027F000FAE30E94F61A80E0809393000091930020
:10280000093018F011F00C944B140091930008302B
:1028100010F00C9424140E94850CA3E9B0E08C9174
:10282000806C87B90E942A1B082F192FA0EFB3E0F4
:10283000FF27E0E10E94361C0E94EE1AE0E7FAE36F
:102840000E94F61A0C9443140091930043E0040F85
:10285000A4E9B0E00C930E94850CF894A0EFB3E0DB
:10286000E4E9F0E0A190BB24ECEEF0E0AA0CBB1C84
:10287000EA0DFB1D0E943E1C0E94EE1AE0E7FAE3FF
:102880000E94F61A7894A3E9B0E08C918F5F8C9344
:1028900011F00C94FE130E94FD1AEAE8FAE30E947C
:1028A000F61A8AE08093930000919300033118F0A8
:1028B00011F00C9478140E944A150E94850CA0E92E
:1028C000B0E08C9183FBA0EFB3E00E94591B8D9385
:1028D00088278C930E94EE1AE0E7FAE30E94F61A2A
:1028E000A3E9B0E08C918F5F8C9311F00C94541499
:1028F0000E94FD1AEEE8FAE30E94F61A84E1809342
:102900009300009193000D3118F011F00C94A51470
:102910000E944A150E94850CA0E9B0E08C9183FBCF
:10292000A0EFB3E00E94591B8D9388278C930E94DF
:10293000EE1AE0E7FAE30E94F61AA3E9B0E08C9100
:102940008F5F8C9311F00C9481140E94FD1AE2E9C0
:10295000FAE30E94F61A80E08093930000919300BE
:10296000093018F011F00C94D2140E944A150E94FC
:10297000850CA0E9B0E08C9183FBA0EFB3E00E944E
:10298000591B8D9388278C930E94EE1AE0E7FAE397
:102990000E94F61AA3E9B0E08C918F5F8C9311F03E
:1029A0000C94AE140E94FD1AE6E9FAE30E94F61AAE
:1029B00088E28093930000919300013318F011F0A6
:1029C0000C940D155A924A9280919300A42DB52D26
:1029D0008C9381E00E94501A0E942506229681E085
:1029E0000E944C1A0E94850CA0E9B0E08C9183FBF8
:1029F000A0EFB3E00E94591B8D9388278C930E940F
:102A0000EE1AE0E7FAE30E94F61AA3E9B0E08C912F
:102A10008F5F8C9311F00C94DB140E94FD1A0C94C0
:102A20004915073011F00C9421150E94850C0E9465
:102A3000681BA7E8B1E00E94F01A0E94FD1A0C94EE
:102A40004915083011F00C9431150E94850C0E9434
:102A5000681BAEE7B1E00E94F01A0E94FD1A0C94C8
:102A60004915093011F00C943E1591E088B3BB274D
:102A7000A8E10E94391B88BB0C9449150A3011F05B
:102A80000C94491591E088B3BB27A8E10E94431B31
:102A900088BB0895A3E9B0E08C919927E5E5F5E1BD
:102AA000880F991FE80FF91F09940C94B9150C941D
:102AB000C4150C94CF150C94DA150C94E5150C94F0
:102AC000F0150C94FB150C9406160C9411160C942E
:102AD0001C160C9427160C9432160C943D160C946C
:102AE00048160C9453160C945E160C9469160C94AC
:102AF00074160C947F160C9499160C94B3160C94BF
:102B0000BE160C94C9160C94D4160C94DF160C94B3
:102B1000EA160C94F5160C9400170C94A5180C9456
:102B2000A5180C940B170C9429170C9447170C94A8
:102B300065170C9483170C94A1170C94BF170C9471
:102B4000DD170C94FB170C9419180C9437180C947F
:102B500042180C944D180C9458180C9463180C944B
:102B60006E180C9479180C9484180C948F180C948B
:102B70009A18A0EAB0E08C9180FBA0E9B0E08C91BB
:102B800083F98C930C94A518A0EAB0E08C9181FB9A
:102B9000A0E9B0E08C9183F98C930C94A518A0EA7D
:102BA000B0E08C9182FBA0E9B0E08C9183F98C932A
:102BB0000C94A518A0EAB0E08C9183FBA0E9B0E0EA
:102BC0008C9183F98C930C94A518A0EAB0E08C91B9
:102BD00084FBA0E9B0E08C9183F98C930C94A51848
:102BE000A0EAB0E08C9185FBA0E9B0E08C9183F97C
:102BF0008C930C94A518A0EAB0E08C9186FBA0E918
:102C0000B0E08C9183F98C930C94A518A0EAB0E005
:102C10008C9187FBA0E9B0E08C9183F98C930C94A4
:102C2000A518A1EAB0E08C9180FBA0E9B0E08C91FE
:102C300083F98C930C94A518A1EAB0E08C9181FBE8
:102C4000A0E9B0E08C9183F98C930C94A518BB2774
:102C5000A0E38C9182FBA0E9B0E08C9183F98C9386
:102C60000C94A518BB27A0E38C9183FBA0E9B0E0EE
:102C70008C9183F98C930C94A518BB27A0E38C91BD
:102C800086FBA0E9B0E08C9183F98C930C94A51895
:102C9000BB27A0E38C9187FBA0E9B0E08C9183F97E
:102CA0008C930C94A518BB27A3E38C9182FBA0E91D
:102CB000B0E08C9183F98C930C94A518BB27A3E307
:102CC0008C9183FBA0E9B0E08C9183F98C930C94F8
:102CD000A518BB27A3E38C9184FBA0E9B0E08C91FD
:102CE00083F98C930C94A518BB27A3E38C9185FBE7
:102CF000A0E9B0E08C9183F98C930C94A5184091D5
:102D000078010091A600041711F40C949216A0E922
:102D1000B0E08C9188608C93809178018093A600BC
:102D20000C949716A0E9B0E08C91877F8C930C945B
:102D3000A518409179010091A700041711F40C9493
:102D4000AC16A0E9B0E08C9188608C9380917901F9
:102D50008093A7000C94B116A0E9B0E08C91877F16
:102D60008C930C94A518BB27A8E38C9180FBA0E959
:102D7000B0E08C9183F98C930C94A518BB27A8E341
:102D80008C9181FBA0E9B0E08C9183F98C930C9439
:102D9000A518BB27A8E38C9182FBA0E9B0E08C9139
:102DA00083F98C930C94A518BB27A8E38C9183FB23
:102DB000A0E9B0E08C9183F98C930C94A518BB2703
:102DC000A8E38C9184FBA0E9B0E08C9183F98C930B
:102DD0000C94A518BB27A8E38C9185FBA0E9B0E073
:102DE0008C9183F98C930C94A518BB27A8E38C9144
:102DF00086FBA0E9B0E08C9183F98C930C94A51824
:102E0000BB27A8E38C9187FBA0E9B0E08C9183F904
:102E10008C930C94A51800274427A2EAB0E08C916B
:102E200080FB00F9A0EAB0E08C9180FB40F9042718
:102E300000FBA0E9B0E08C9183F98C93A0EAB0E0AC
:102E40008C9180FBA2EAB0E08C9180F98C930C9479
:102E5000A51800274427A2EAB0E08C9181FB00F975
:102E6000A0EAB0E08C9181FB40F9042700FBA0E9C7
:102E7000B0E08C9183F98C93A0EAB0E08C9181FB57
:102E8000A2EAB0E08C9181F98C930C94A5180027EC
:102E90004427A2EAB0E08C9182FB00F9A0EAB0E0FE
:102EA0008C9182FB40F9042700FBA0E9B0E08C91F3
:102EB00083F98C93A0EAB0E08C9182FBA2EAB0E0A7
:102EC0008C9182F98C930C94A51800274427A2EAD0
:102ED000B0E08C9183FB00F9A0EAB0E08C9183FB19
:102EE00040F9042700FBA0E9B0E08C9183F98C93B2
:102EF000A0EAB0E08C9183FBA2EAB0E08C9183F968
:102F00008C930C94A51800274427A2EAB0E08C917A
:102F100084FB00F9A0EAB0E08C9184FB40F904271F
:102F200000FBA0E9B0E08C9183F98C93A0EAB0E0BB
:102F30008C9184FBA2EAB0E08C9184F98C930C9480
:102F4000A51800274427A2EAB0E08C9185FB00F980
:102F5000A0EAB0E08C9185FB40F9042700FBA0E9D2
:102F6000B0E08C9183F98C93A0EAB0E08C9185FB62
:102F7000A2EAB0E08C9185F98C930C94A5180027F7
:102F80004427A2EAB0E08C9186FB00F9A0EAB0E009
:102F90008C9186FB40F9042700FBA0E9B0E08C91FE
:102FA00083F98C93A0EAB0E08C9186FBA2EAB0E0B2
:102FB0008C9186F98C930C94A51800274427A2EADB
:102FC000B0E08C9187FB00F9A0EAB0E08C9187FB20
:102FD00040F9042700FBA0E9B0E08C9183F98C93C1
:102FE000A0EAB0E08C9187FBA2EAB0E08C9187F96F
:102FF0008C930C94A51800274427A3EAB0E08C9189
:1030000080FB00F9A1EAB0E08C9180FB40F9042735
:1030100000FBA0E9B0E08C9183F98C93A1EAB0E0C9
:103020008C9180FBA3EAB0E08C9180F98C930C9496
:10303000A51800274427A3EAB0E08C9181FB00F992
:10304000A1EAB0E08C9181FB40F9042700FBA0E9E4
:10305000B0E08C9183F98C93A1EAB0E08C9181FB74
:10306000A3EAB0E08C9181F98C930C94A518A4EAA2
:10307000B0E08C9180FBA0E9B0E08C9183F98C9357
:103080000C94A518A4EAB0E08C9181FBA0E9B0E013
:103090008C9183F98C930C94A518A4EAB0E08C91E0
:1030A00082FBA0E9B0E08C9183F98C930C94A51875
:1030B000A4EAB0E08C9183FBA0E9B0E08C9183F9A5
:1030C0008C930C94A518A4EAB0E08C9184FBA0E941
:1030D000B0E08C9183F98C930C94A518A4EAB0E02D
:1030E0008C9185FBA0E9B0E08C9183F98C930C94D2
:1030F000A518A4EAB0E08C9186FBA0E9B0E08C9121
:1031000083F98C930C94A518A4EAB0E08C9187FB0A
:10311000A0E9B0E08C9183F98C930C94A518A5EAF2
:10312000B0E08C9180FBA0E9B0E08C9183F98C93A6
:103130000C94A518A5EAB0E08C9181FBA0E9B0E061
:103140008C9183F98C930C94A5180895A3E9B0E0B1
:103150008C919927E1EBF8E1880F991FE80FF91F8F
:1031600009940C9415190C9420190C942B190C9497
:1031700036190C9441190C944C190C9457190C9451
:1031800062190C946D190C9478190C94491A0C94CA
:10319000491A0C94491A0C94491A0C94491A0C9423
:1031A000491A0C94491A0C94491A0C94491A0C9413
:1031B000491A0C9483190C948E190C9499190C9437
:1031C000A4190C94AF190C94BA190C94C5190C9449
:1031D000D0190C94491A0C94491A0C94491A0C945D
:1031E000491A0C94491A0C94491A0C94491A0C94D3
:1031F000491A0C94491A0C94491A0C94491A0C94C3
:10320000491A0C94DB190C94E6190C94F1190C94DE
:10321000FC190C94071A0C94121A0C941D1A0C9495
:10322000281A0C94331A0C943E1AA0E9B0E08C9141
:1032300083FBA0EAB0E08C9180F98C930C94491A3E
:10324000A0E9B0E08C9183FBA0EAB0E08C9181F919
:103250008C930C94491AA0E9B0E08C9183FBA0EA0E
:10326000B0E08C9182F98C930C94491AA0E9B0E0FB
:103270008C9183FBA0EAB0E08C9183F98C930C9441
:10328000491AA0E9B0E08C9183FBA0EAB0E08C91F0
:1032900084F98C930C94491AA0E9B0E08C9183FBDB
:1032A000A0EAB0E08C9185F98C930C94491AA0E9BE
:1032B000B0E08C9183FBA0EAB0E08C9186F98C930E
:1032C0000C94491AA0E9B0E08C9183FBA0EAB0E02D
:1032D0008C9187F98C930C94491AA0E9B0E08C91F9
:1032E00083FBA1EAB0E08C9180F98C930C94491A8D
:1032F000A0E9B0E08C9183FBA1EAB0E08C9181F968
:103300008C930C94491AA0E9B0E08C9183FBBB2705
:10331000A8E38C9180F98C930C94491AA0E9B0E051
:103320008C9183FBBB27A8E38C9181F98C930C943F
:10333000491AA0E9B0E08C9183FBBB27A8E38C91EC
:1033400082F98C930C94491AA0E9B0E08C9183FB2C
:10335000BB27A8E38C9183F98C930C94491AA0E9BC
:10336000B0E08C9183FBBB27A8E38C9184F98C930C
:103370000C94491AA0E9B0E08C9183FBBB27A8E329
:103380008C9185F98C930C94491AA0E9B0E08C914A
:1033900083FBBB27A8E38C9186F98C930C94491A84
:1033A000A0E9B0E08C9183FBBB27A8E38C9187F95F
:1033B0008C930C94491AA0E9B0E08C9183FBA4EAA9
:1033C000B0E08C9180F98C930C94491AA0E9B0E09C
:1033D0008C9183FBA4EAB0E08C9181F98C930C94DE
:1033E000491AA0E9B0E08C9183FBA4EAB0E08C918B
:1033F00082F98C930C94491AA0E9B0E08C9183FB7C
:10340000A4EAB0E08C9183F98C930C94491AA0E95A
:10341000B0E08C9183FBA4EAB0E08C9184F98C93AA
:103420000C94491AA0E9B0E08C9183FBA4EAB0E0C7
:103430008C9185F98C930C94491AA0E9B0E08C9199
:1034400083FBA4EAB0E08C9186F98C930C94491A22
:10345000A0E9B0E08C9183FBA4EAB0E08C9187F9FD
:103460008C930C94491AA0E9B0E08C9183FBA5EAF7
:10347000B0E08C9180F98C930C94491AA0E9B0E0EB
:103480008C9183FBA5EAB0E08C9181F98C930C942C
:10349000491A0895F894FFCF481A8827580A0895C2
:1034A000480E8827581E0895ED91FC913197FC93A2
:1034B000EE93089508D03DD000FC10D0089503D0BD
:1034C0001ED001F8F9CF0024E89457FF02C009D0BC
:1034D000689400F80BD010F80124089502D009D0A8
:1034E0000895509540954F5F5F4F0895E89417FFFA
:1034F0000895009510950F5F1F4F68940895352F1C
:10350000242FE894452B11F468940895512F402FEF
:103510000027112780E1440F551F001F111F021BB8
:10352000130B416018F4020F131F4E7F8A9599F711
:103530000895752F642F55274427FF93F1E1889450
:1035400005C010F4460F571F5695479517950795D8
:10355000FA95B9F7FF910895C8950D92319600201C
:10356000D9F7089581918D938823E1F708958F937A
:103570008D918823E9F711978F910895919199235F
:1035800051F08A95D9F7319781918D930A9519F069
:103590008823D1F7089588278D9308958091750128
:1035A000803009F001C00895AF93BF93A5E7B1E063
:1035B0008C918823E9F38A958D9311968C918E31A5
:1035C00008F0882783958C93A6E5B1E0A80F88279B
:1035D000B81F11978C91BF91AF910895A0EFB3E000
:1035E0008D91882311F00CD0FBCF08950E944D1BC4
:1035F000802D11F005D0FACF08958DE001D08AE03A
:10360000F8949F93AF93BF9390915301923398F4A2
:1036100093959093530190915401A0E2B1E0A90FCA
:103620009F939927B91F8C939F91923308F0992704
:10363000939590935401BF91AF919F91559A78942F
:1036400008953197F1F70895689462F80895E89421
:1036500062F80895369A3699FECF369A3699FECF9B
:1036600084B195B108955A924A92480E8827581EFF
:103670000895903039F08C91880F08F481609A9504
:10368000D9F78C930895903039F08C91869508F491
:1036900080689A95D9F78C930895C8953196002043
:1036A000089582E001C084E099279D938A95E9F707
:1036B000089580E30EF48395089500278A3018F06A
:1036C0008A500395FBCF005D0D93805D8D93089527
:1036D000AEE7B1E0ECE7F1E08081EFDF8FE28D93C0
:1036E0008291EBDF8FE28D9332968081E6DF88272F
:1036F0008D9332978291E1DF8AE38D938291DDDFB2
:103700008AE38D938291D9DF88278C930895AF93B4
:10371000BF930F939F938F938FB78F93A8E7B1E0D9
:103720008C9183958D938C3309F03DC088278E93BF
:1037300011968C9183958D938C3309F034C0882732
:103740008E9311968C9183958D93883161F588279E
:103750008E9311968C9183958D939C910EE194306C
:1037600089F0963079F0993069F09B3059F00CE18E
:10377000923039F411969C911197937019F4039536
:1037800001C00FE1801778F071F081E08E931196FF
:103790008C9183958D938D3031F481E08E931196C9
:1037A0008C9183958C938F918FBF8F919F910F9167
:1037B000BF91AF911895AF93BF938F939F938FB79E
:1037C0008F93A5E7B1E09C919E3180F493959D93F2
:1037D0009C919E3108F0992793959C93A6E5B1E0C2
:1037E000A90F9927B91F11978CB18C938F918FBF17
:1037F0009F918F91BF91AF9118958F938FB78F93B2
:103800009F93AF93BF93A3E5B1E09C91992311F4EB
:10381000559812C09A959C9312969C91A0E2B1E0A3
:10382000A90F8827B81F8C91923308F09927939598
:10383000A5E5B1E09C938CB9BF91AF919F918F9119
:103840008FBF8F911895040F151F261F371F0895DE
:10385000000F111F221F331F08950095109520950A
:1038600030950F5F1F4F2F4F3F4F089501911081EB
:103870000EC001911191219130810BC001911081F5
:1038800017FF05C03FEF2FEF04C00081112722274B
:10389000332737FF03C0E1DF8DE28D93CF93DF93B2
:1038A000AA24BB24CC24DD24EE2440E2CAE0DD2798
:1038B00055E093E38881890F87FD9F7083FD907F9A
:1038C000891B89935A95A9F7C3DFAA1CBB1CCC1C82
:1038D000DD1CEE1C4A9551F7E894EFE0FF2782913A
:1038E0000BD0EB30E0F71EF068948A2D09D08827C2
:1038F0008D93DF91CF9108958F93829501D08F9111
:103900008F70805D26F0803309F4089568948D935C
:10391000089500271127222733271DD08A3328F442
:10392000803318F005D015D0F9CF0EF496CF089556
:1039300080538F93402F512F622F732F89DF88DFA1
:1039400082DF86DF8F919927080F191F291F391FE2
:1039500008958D910895E894FCDF8032E9F3893071
:10396000D9F38D3211F46894F4CF0895E199FECF24
:10397000EEBBFFBB3196089591E001C092E0F6DF07
:103980008D918DBBE29AE19A9A95C9F70895EEDF81
:103990008D918DBBE29AE19A8823C9F7089591E051
:1039A00001C092E0E3DFE09A8DB38D939A95D1F751
:1039B0000895DCDFE09A8DB38D938823D1F70895C5
:1039C0008FEF83959D919923E1F70895689401C045
:1039D000E894AF93BF938D9116F0919103C00E942C
:1039E0004D1B902D891718F011F48823A1F7BF9172
:1039F000AF91089520002A002B002D002F005C00BD
:103A00003E003C005D006332000072003D00730028
:103A10007000750074006500660062004200690075
:103A200049006F004F0064006800480063302D6853
:103A30006C70202063312D707267000063322D732B
:103A40007470202063332D72756E000063342D6C0A
:103A50007374202063352D76616C000063362D74FD
:103A6000696D202063372D6461740000723D000091
:103A70002C00733D0000653D0000663D0000743D74
:103A80000000703D0000753D0000693D00006F3D85
:0A3A90000000623D0000683D0000E8
:00000001FF
